HI-TECH Software C Compiler 

Linker command line:

--edf=C:\Program Files (x86)\HI-TECH Software\PICC\9.83\dat\en_msgs.txt -cs \
  -h+Zadatak 4..sym -z -Q16F690 -ol.obj -MZadatak 4..map -E1 \
  -ACONST=00h-0FFhx16 -ACODE=00h-07FFhx2 -ASTRCODE=00h-0FFFh \
  -AENTRY=00h-0FFhx16 -ASTRING=00h-0FFhx16 -ABANK0=020h-06Fh \
  -ABANK1=0A0h-0EFh -ABANK2=0120h-016Fh \
  -ARAM=020h-06Fh,0A0h-0EFh,0120h-016Fh \
  -AABS1=020h-07Fh,0A0h-0EFh,0120h-016Fh -ACOMMON=070h-07Fh -ASFR0=00h-01Fh \
  -ASFR1=080h-09Fh -ASFR2=0100h-011Fh -ASFR3=0180h-01EFh \
  -preset_vec=00h,intentry,init,end_init -ppowerup=CODE -pfunctab=CODE \
  -ACONFIG=02007h-02007h -pconfig=CONFIG -DCONFIG=2 -AIDLOC=02000h-02003h \
  -pidloc=IDLOC -DIDLOC=2 -AEEDATA=00h-0FFh/02100h -peeprom_data=EEDATA \
  -DEEDATA=2 -DCODE=2 -DSTRCODE=2 -DSTRING=2 -DCONST=2 -DENTRY=2 -k \
  startup.obj Zadatak 4..obj 

Object code version is 3.10

Machine type is 16F690



                Name                               Link     Load   Length Selector   Space Scale
startup.obj     end_init                              0        0        2        0       0
Zadatak 4..obj  config                             2007     2007        1     400E       0
                text674                             A85      A85       12     150A       0
                text673                             A67      A67        E     14CE       0
                text672                             ABB      ABB       14     1576       0
                text671                             DF7      DF7       7B     1BEE       0
                text670                             E72      E72       A4     1CE4       0
                text669                             D81      D81       76     1B02       0
                text668                             CB5      CB5       66     196A       0
                text667                             ACF      ACF       14     159E       0
                text666                             A75      A75       10     14EA       0
                text665                             AF8      AF8       17     15F0       0
                text664                             A97      A97       12     152E       0
                text663                             B6F      B6F       30     16DE       0
                text662                             B9F      B9F       33     173E       0
                text661                               5        5       C4        A       0
                text660                             F16      F16       EA     1E2C       0
                text659                             AE3      AE3       15     15C6       0
                text658                             C19      C19       4E     1832       0
                text657                             B29      B29       20     1652       0
                text656                             C67      C67       4E     18CE       0
                text655                              C9       C9      18A      192       0
                text654                             253      253      18A      4A6       0
                text653                             3DD      3DD      18A      7BA       0
                text652                             A5C      A5C        B     14B8       0
                text651                             AA9      AA9       12     1552       0
                text650                             B49      B49       26     1692       0
                text649                             B0F      B0F       1A     161E       0
                text648                             BD2      BD2       47     17A4       0
                text647                             D1B      D1B       66     1A36       0
                maintext                            567      567      299      ACE       0
                cstackBANK0                          20       20       27       20       1
                cstackCOMMON                         70       70        E       70       1
                cinit                                 2        2        3        0       0
                stringtext                          800      800      12E       10       0
                strings                             92E      92E       12     125C       0

TOTAL           Name                               Link     Load   Length     Space
        CLASS   CONST          

        CLASS   CODE           
                end_init                              0        0        2         0
                text674                             A85      A85       12         0
                text673                             A67      A67        E         0
                text672                             ABB      ABB       14         0
                text671                             DF7      DF7       7B         0
                text670                             E72      E72       A4         0
                text669                             D81      D81       76         0
                text668                             CB5      CB5       66         0
                text667                             ACF      ACF       14         0
                text666                             A75      A75       10         0
                text665                             AF8      AF8       17         0
                text664                             A97      A97       12         0
                text663                             B6F      B6F       30         0
                text662                             B9F      B9F       33         0
                text661                               5        5       C4         0
                text660                             F16      F16       EA         0
                text659                             AE3      AE3       15         0
                text658                             C19      C19       4E         0
                text657                             B29      B29       20         0
                text656                             C67      C67       4E         0
                text655                              C9       C9      18A         0
                text654                             253      253      18A         0
                text653                             3DD      3DD      18A         0
                text652                             A5C      A5C        B         0
                text651                             AA9      AA9       12         0
                text650                             B49      B49       26         0
                text649                             B0F      B0F       1A         0
                text648                             BD2      BD2       47         0
                text647                             D1B      D1B       66         0
                maintext                            567      567      299         0
                cinit                                 2        2        3         0

        CLASS   STRCODE        
                stringtext                          800      800      12E         0

        CLASS   ENTRY          

        CLASS   STRING         
                strings                             92E      92E       12         0

        CLASS   BANK0          
                cstackBANK0                          20       20       27         1

        CLASS   BANK1          

        CLASS   BANK2          

        CLASS   RAM            

        CLASS   ABS1           
                abs_s1                               7E       7E        2         1

        CLASS   COMMON         
                cstackCOMMON                         70       70        E         1

        CLASS   SFR0           

        CLASS   SFR1           

        CLASS   SFR2           

        CLASS   SFR3           

        CLASS   CONFIG         
                config                             2007     2007        1         0

        CLASS   IDLOC          

        CLASS   EEDATA         

        CLASS   BANK3          



SEGMENTS        Name                           Load    Length   Top    Selector   Space  Class     Delta

                reset_vec                      000000  000005  000005         0       0  CODE        2
                text661                        000005  0000C4  0000C9         A       0  CODE        2
                cstackBANK0                    000020  000027  000047        20       1  BANK0       1
                cstackCOMMON                   000070  00000E  00007E        70       1  COMMON      1
                text655                        0000C9  00018A  000253       192       0  CODE        2
                text654                        000253  00018A  0003DD       4A6       0  CODE        2
                text653                        0003DD  00018A  000567       7BA       0  CODE        2
                maintext                       000567  000299  000800       ACE       0  CODE        2
                stringtext                     000800  00012E  00092E        10       0  STRCODE     2
                strings                        00092E  000012  000940      125C       0  STRING      2
                text652                        000A5C  00000B  000A67      14B8       0  CODE        2
                text673                        000A67  00000E  000A75      14CE       0  CODE        2
                text666                        000A75  000010  000A85      14EA       0  CODE        2
                text674                        000A85  000012  000A97      150A       0  CODE        2
                text664                        000A97  000012  000AA9      152E       0  CODE        2
                text651                        000AA9  000012  000ABB      1552       0  CODE        2
                text672                        000ABB  000014  000ACF      1576       0  CODE        2
                text667                        000ACF  000014  000AE3      159E       0  CODE        2
                text659                        000AE3  000015  000AF8      15C6       0  CODE        2
                text665                        000AF8  000017  000B0F      15F0       0  CODE        2
                text649                        000B0F  00001A  000B29      161E       0  CODE        2
                text657                        000B29  000020  000B49      1652       0  CODE        2
                text650                        000B49  000026  000B6F      1692       0  CODE        2
                text663                        000B6F  000030  000B9F      16DE       0  CODE        2
                text662                        000B9F  000033  000BD2      173E       0  CODE        2
                text648                        000BD2  000047  000C19      17A4       0  CODE        2
                text658                        000C19  00004E  000C67      1832       0  CODE        2
                text656                        000C67  00004E  000CB5      18CE       0  CODE        2
                text668                        000CB5  000066  000D1B      196A       0  CODE        2
                text647                        000D1B  000066  000D81      1A36       0  CODE        2
                text669                        000D81  000076  000DF7      1B02       0  CODE        2
                text671                        000DF7  00007B  000E72      1BEE       0  CODE        2
                text670                        000E72  0000A4  000F16      1CE4       0  CODE        2
                text660                        000F16  0000EA  001000      1E2C       0  CODE        2
                config                         002007  000001  002008      400E       0  CONFIG      2


UNUSED ADDRESS RANGES

        Name                Unused          Largest block    Delta
        BANK0            0047-006F             29           1
        BANK1            00A0-00EF             50           1
        BANK2            0120-016F             50           1
        CODE             0940-0A5B            11C           2
        CONST            0940-0A5B             C0           2
        EEDATA           2100-21FF            100           2
        ENTRY            0940-0A5B             C0           2
        IDLOC            2000-2003              4           2
        RAM              0047-006F             29           1
                         00A0-00EF             50
                         0120-016F             50
        SFR0             0000-001F             20           1
        SFR1             0080-009F             20           1
        SFR2             0100-011F             20           1
        SFR3             0180-01EF             70           1
        STRCODE          0940-0A5B            11C           2
        STRING           0940-0A5B             C0           2

                                  Symbol Table

??___awdiv                 cstackCOMMON 007B
??___awmod                 cstackCOMMON 0074
??___ftdiv                 cstackBANK0  0020
??___ftmul                 cstackBANK0  0020
??___ftpack                cstackCOMMON 0075
??___fttol                 cstackCOMMON 0074
??___lwtoft                cstackCOMMON 007B
??_acc_skaliranje          cstackBANK0  002B
??_gyro_skaliranje         cstackBANK0  002B
??_i2c_get_byte            cstackCOMMON 0078
??_i2c_init                cstackCOMMON 007B
??_i2c_open                cstackCOMMON 0077
??_i2c_put_byte            cstackCOMMON 0074
??_i2c_read_ack            cstackCOMMON 0071
??_i2c_read_byte           cstackCOMMON 0071
??_i2c_restart             cstackCOMMON 0070
??_i2c_send_ack            cstackCOMMON 0070
??_i2c_send_address        cstackCOMMON 0075
??_i2c_send_byte           cstackCOMMON 0071
??_i2c_stop                cstackCOMMON 0070
??_i2c_wait_for_SCL        cstackCOMMON 0070
??_init_PIC                cstackCOMMON 0070
??_mag_skaliranje          cstackBANK0  002B
??_main                    cstackBANK0  0042
??_read_i2c                cstackBANK0  0022
??_rs232_init              cstackCOMMON 0070
??_rs232_send_byte         cstackCOMMON 0070
??_rs232_send_text         cstackCOMMON 0073
??_start                   cstackCOMMON 0072
?___awdiv                  cstackCOMMON 0077
?___awmod                  cstackCOMMON 0070
?___ftdiv                  cstackCOMMON 0078
?___ftmul                  cstackCOMMON 0078
?___ftpack                 cstackCOMMON 0070
?___fttol                  cstackCOMMON 0070
?___lwtoft                 cstackCOMMON 0078
?_acc_skaliranje           cstackBANK0  002A
?_gyro_skaliranje          cstackBANK0  002A
?_i2c_get_byte             cstackCOMMON 0076
?_i2c_init                 cstackCOMMON 0079
?_i2c_open                 cstackCOMMON 0076
?_i2c_put_byte             cstackCOMMON 0070
?_i2c_read_ack             cstackCOMMON 0070
?_i2c_read_byte            cstackCOMMON 0070
?_i2c_restart              cstackCOMMON 0070
?_i2c_send_ack             cstackCOMMON 0070
?_i2c_send_address         cstackCOMMON 0074
?_i2c_send_byte            cstackCOMMON 0070
?_i2c_stop                 cstackCOMMON 0070
?_i2c_wait_for_SCL         cstackCOMMON 0070
?_init_PIC                 cstackCOMMON 0070
?_mag_skaliranje           cstackBANK0  002A
?_main                     cstackCOMMON 0070
?_read_i2c                 cstackBANK0  0020
?_rs232_init               cstackCOMMON 0070
?_rs232_send_byte          cstackCOMMON 0070
?_rs232_send_text          cstackCOMMON 0071
?_start                    cstackCOMMON 0070
_ANSEL                     (abs)        011E
_ANSELH                    (abs)        011F
_CARRY                     (abs)        0018
_CREN                      (abs)        00C4
_EEADR                     (abs)        010D
_EECON1                    (abs)        018C
_EECON2                    (abs)        018D
_EEDATA                    (abs)        010C
_FERR                      (abs)        00C2
_GIE                       (abs)        005F
_OERR                      (abs)        00C1
_PORTA                     (abs)        0005
_PORTB                     (abs)        0006
_PORTC                     (abs)        0007
_RA3                       (abs)        002B
_RB4                       (abs)        0034
_RB6                       (abs)        0036
_RCIF                      (abs)        0065
_RCREG                     (abs)        001A
_RCSTA                     (abs)        0018
_RD                        (abs)        0C60
_SPBRG                     (abs)        0099
_SSPCON                    (abs)        0014
_TRISA                     (abs)        0085
_TRISB                     (abs)        0086
_TRISB4                    (abs)        0434
_TRISB6                    (abs)        0436
_TRISC                     (abs)        0087
_TRMT                      (abs)        04C1
_TXREG                     (abs)        0019
_TXSTA                     (abs)        0098
_WR                        (abs)        0C61
_WREN                      (abs)        0C62
__Habs1                    abs1         0000
__Hbank0                   bank0        0000
__Hbank1                   bank1        0000
__Hbank2                   bank2        0000
__Hbank3                   bank3        0000
__Hcinit                   cinit        0000
__Hclrtext                 clrtext      0000
__Hcode                    code         0000
__Hcommon                  common       0000
__Hconfig                  config       2008
__HcstackBANK0             cstackBANK0  0000
__HcstackCOMMON            cstackCOMMON 0000
__Heeprom_data             eeprom_data  0000
__Hend_init                end_init     0002
__Hfunctab                 functab      0000
__Hidloc                   idloc        0000
__Hinit                    init         0000
__Hintentry                intentry     0000
__Hmaintext                maintext     0000
__Hpowerup                 powerup      0000
__Hram                     ram          0000
__Hreset_vec               reset_vec    0000
__Hsfr0                    sfr0         0000
__Hsfr1                    sfr1         0000
__Hsfr2                    sfr2         0000
__Hsfr3                    sfr3         0000
__Hstrings                 strings      0000
__Hstringtext              stringtext   0000
__Htext                    text         0000
__Labs1                    abs1         0000
__Lbank0                   bank0        0000
__Lbank1                   bank1        0000
__Lbank2                   bank2        0000
__Lbank3                   bank3        0000
__Lcinit                   cinit        0000
__Lclrtext                 clrtext      0000
__Lcode                    code         0000
__Lcommon                  common       0000
__Lconfig                  config       2007
__LcstackBANK0             cstackBANK0  0000
__LcstackCOMMON            cstackCOMMON 0000
__Leeprom_data             eeprom_data  0000
__Lend_init                end_init     0000
__Lfunctab                 functab      0000
__Lidloc                   idloc        0000
__Linit                    init         0000
__Lintentry                intentry     0000
__Lmaintext                maintext     0000
__Lpowerup                 powerup      0000
__Lram                     ram          0000
__Lreset_vec               reset_vec    0000
__Lsfr0                    sfr0         0000
__Lsfr1                    sfr1         0000
__Lsfr2                    sfr2         0000
__Lsfr3                    sfr3         0000
__Lstrings                 strings      0000
__Lstringtext              stringtext   0000
__Ltext                    text         0000
__S0                       (abs)        2008
__S1                       (abs)        007E
__S2                       (abs)        0000
___awdiv                   text669      0D81
___awdiv@counter           cstackBANK0  0020
___awdiv@dividend          cstackCOMMON 0079
___awdiv@divisor           cstackCOMMON 0077
___awdiv@quotient          cstackBANK0  0022
___awdiv@sign              cstackBANK0  0021
___awmod                   text668      0CB5
___awmod@counter           cstackCOMMON 0075
___awmod@dividend          cstackCOMMON 0072
___awmod@divisor           cstackCOMMON 0070
___awmod@sign              cstackCOMMON 0076
___ftdiv                   text661      0005
___ftdiv@cntr              cstackBANK0  0024
___ftdiv@exp               cstackBANK0  0028
___ftdiv@f1                cstackCOMMON 007B
___ftdiv@f2                cstackCOMMON 0078
___ftdiv@f3                cstackBANK0  0025
___ftdiv@sign              cstackBANK0  0029
___ftmul                   text660      0F16
___ftmul@cntr              cstackBANK0  0028
___ftmul@exp               cstackBANK0  0024
___ftmul@f1                cstackCOMMON 0078
___ftmul@f2                cstackCOMMON 007B
___ftmul@f3_as_product     cstackBANK0  0025
___ftmul@sign              cstackBANK0  0029
___ftpack                  text671      0DF7
___ftpack@arg              cstackCOMMON 0070
___ftpack@exp              cstackCOMMON 0073
___ftpack@sign             cstackCOMMON 0074
___fttol                   text670      0E72
___fttol@exp1              cstackCOMMON 007D
___fttol@f1                cstackCOMMON 0070
___fttol@lval              cstackCOMMON 0079
___fttol@sign1             cstackCOMMON 0078
___lwtoft                  text659      0AE3
___lwtoft@c                cstackCOMMON 0078
__end_of___awdiv           text669      0DF7
__end_of___awmod           text668      0D1B
__end_of___ftdiv           text661      00C9
__end_of___ftmul           text660      1000
__end_of___ftpack          text671      0E72
__end_of___fttol           text670      0F16
__end_of___lwtoft          text659      0AF8
__end_of_acc_skaliranje    text655      0253
__end_of_gyro_skaliranje   text654      03DD
__end_of_i2c_get_byte      text650      0B6F
__end_of_i2c_init          text648      0C19
__end_of_i2c_open          text649      0B29
__end_of_i2c_put_byte      text651      0ABB
__end_of_i2c_read_ack      text657      0B49
__end_of_i2c_read_byte     text656      0CB5
__end_of_i2c_restart       text666      0A85
__end_of_i2c_send_ack      text664      0AA9
__end_of_i2c_send_address  text652      0A67
__end_of_i2c_send_byte     text658      0C67
__end_of_i2c_stop          text667      0AE3
__end_of_i2c_wait_for_SCL  text665      0B0F
__end_of_init_PIC          text672      0ACF
__end_of_mag_skaliranje    text653      0567
__end_of_main              maintext     0800
__end_of_read_i2c          text647      0D81
__end_of_rs232_init        text674      0A97
__end_of_rs232_send_byte   text673      0A75
__end_of_rs232_send_text   text663      0B9F
__end_of_start             text662      0BD2
__pcstackBANK0             cstackBANK0  0020
__pcstackCOMMON            cstackCOMMON 0070
__pmaintext                maintext     0567
__pstrings                 strings      092E
__pstringtext              stringtext   0800
__ptext646                 text646      0000
__ptext647                 text647      0D1B
__ptext648                 text648      0BD2
__ptext649                 text649      0B0F
__ptext650                 text650      0B49
__ptext651                 text651      0AA9
__ptext652                 text652      0A5C
__ptext653                 text653      03DD
__ptext654                 text654      0253
__ptext655                 text655      00C9
__ptext656                 text656      0C67
__ptext657                 text657      0B29
__ptext658                 text658      0C19
__ptext659                 text659      0AE3
__ptext660                 text660      0F16
__ptext661                 text661      0005
__ptext662                 text662      0B9F
__ptext663                 text663      0B6F
__ptext664                 text664      0A97
__ptext665                 text665      0AF8
__ptext666                 text666      0A75
__ptext667                 text667      0ACF
__ptext668                 text668      0CB5
__ptext669                 text669      0D81
__ptext670                 text670      0E72
__ptext671                 text671      0DF7
__ptext672                 text672      0ABB
__ptext673                 text673      0A67
__ptext674                 text674      0A85
__ptext675                 text675      0000
__size_of___awdiv          (abs)        0000
__size_of___awmod          (abs)        0000
__size_of___ftdiv          (abs)        0000
__size_of___ftmul          (abs)        0000
__size_of___ftpack         (abs)        0000
__size_of___fttol          (abs)        0000
__size_of___lwtoft         (abs)        0000
__size_of_acc_skaliranje   (abs)        0000
__size_of_gyro_skaliranje  (abs)        0000
__size_of_i2c_get_byte     (abs)        0000
__size_of_i2c_init         (abs)        0000
__size_of_i2c_open         (abs)        0000
__size_of_i2c_put_byte     (abs)        0000
__size_of_i2c_read_ack     (abs)        0000
__size_of_i2c_read_byte    (abs)        0000
__size_of_i2c_restart      (abs)        0000
__size_of_i2c_send_ack     (abs)        0000
__size_of_i2c_send_address (abs)        0000
__size_of_i2c_send_byte    (abs)        0000
__size_of_i2c_stop         (abs)        0000
__size_of_i2c_wait_for_SCL (abs)        0000
__size_of_init_PIC         (abs)        0000
__size_of_mag_skaliranje   (abs)        0000
__size_of_main             (abs)        0000
__size_of_read_i2c         (abs)        0000
__size_of_rs232_init       (abs)        0000
__size_of_rs232_send_byte  (abs)        0000
__size_of_rs232_send_text  (abs)        0000
__size_of_start            (abs)        0000
_acc_skaliranje            text655      00C9
_exit                      init         0000
_gyro_skaliranje           text654      0253
_i2c_get_byte              text650      0B49
_i2c_init                  text648      0BD2
_i2c_open                  text649      0B0F
_i2c_put_byte              text651      0AA9
_i2c_read_ack              text657      0B29
_i2c_read_byte             text656      0C67
_i2c_restart               text666      0A75
_i2c_send_ack              text664      0A97
_i2c_send_address          text652      0A5C
_i2c_send_byte             text658      0C19
_i2c_stop                  text667      0ACF
_i2c_wait_for_SCL          text665      0AF8
_init_PIC                  text672      0ABB
_mag_skaliranje            text653      03DD
_main                      maintext     0567
_read_i2c                  text647      0D1B
_rs232_init                text674      0A85
_rs232_send_byte           text673      0A67
_rs232_send_text           text663      0B6F
_start                     text662      0B9F
acc_skaliranje@d           cstackBANK0  0038
acc_skaliranje@dt          cstackBANK0  0032
acc_skaliranje@high        cstackBANK0  003C
acc_skaliranje@high_int    cstackBANK0  002D
acc_skaliranje@j           cstackBANK0  003A
acc_skaliranje@low         cstackBANK0  002A
acc_skaliranje@low_int     cstackBANK0  002F
acc_skaliranje@mask        cstackBANK0  0031
acc_skaliranje@rez         cstackBANK0  003D
acc_skaliranje@s           cstackBANK0  0036
acc_skaliranje@t           cstackBANK0  0034
acc_skaliranje@temp        cstackBANK0  0040
btemp                      (abs)        007E
end_of_initialization      cinit        0002
gyro_skaliranje@d          cstackBANK0  0038
gyro_skaliranje@dt         cstackBANK0  0032
gyro_skaliranje@high       cstackBANK0  003C
gyro_skaliranje@high_int   cstackBANK0  002D
gyro_skaliranje@j          cstackBANK0  003A
gyro_skaliranje@low        cstackBANK0  002A
gyro_skaliranje@low_int    cstackBANK0  002F
gyro_skaliranje@mask       cstackBANK0  0031
gyro_skaliranje@rez        cstackBANK0  003D
gyro_skaliranje@s          cstackBANK0  0036
gyro_skaliranje@t          cstackBANK0  0034
gyro_skaliranje@temp       cstackBANK0  0040
i2c_get_byte@byte          cstackCOMMON 007A
i2c_get_byte@more          cstackCOMMON 007C
i2c_init@ADRESA1           cstackCOMMON 007B
i2c_init@ADRESA2           cstackCOMMON 0079
i2c_init@ADRESA3           cstackCOMMON 007A
i2c_open@address           cstackCOMMON 0078
i2c_open@mode              cstackCOMMON 0076
i2c_put_byte@data          cstackCOMMON 0074
i2c_read_ack@ack           cstackCOMMON 0072
i2c_read_byte@byte         cstackCOMMON 0075
i2c_read_byte@i            cstackCOMMON 0073
i2c_send_ack@status        cstackCOMMON 0070
i2c_send_address@address   cstackCOMMON 0075
i2c_send_address@rw        cstackCOMMON 0074
i2c_send_byte@byte         cstackCOMMON 0072
i2c_send_byte@i            cstackCOMMON 0073
intlevel0                  functab      0000
intlevel1                  functab      0000
intlevel2                  functab      0000
intlevel3                  functab      0000
intlevel4                  functab      0000
intlevel5                  functab      0000
mag_skaliranje@d           cstackBANK0  0038
mag_skaliranje@dt          cstackBANK0  0032
mag_skaliranje@high        cstackBANK0  003C
mag_skaliranje@high_int    cstackBANK0  002D
mag_skaliranje@j           cstackBANK0  003A
mag_skaliranje@low         cstackBANK0  002A
mag_skaliranje@low_int     cstackBANK0  002F
mag_skaliranje@mask        cstackBANK0  0031
mag_skaliranje@rez         cstackBANK0  003D
mag_skaliranje@s           cstackBANK0  0036
mag_skaliranje@t           cstackBANK0  0034
mag_skaliranje@temp        cstackBANK0  0040
main@high                  cstackBANK0  0045
main@low                   cstackBANK0  0046
read_i2c@ADRESA            cstackBANK0  0025
read_i2c@adr_reg           cstackBANK0  0020
read_i2c@data              cstackBANK0  0024
reset_vec                  reset_vec    0000
rs232_send_byte@x          cstackCOMMON 0070
rs232_send_text@c          cstackCOMMON 0074
rs232_send_text@i          cstackCOMMON 0075
rs232_send_text@string     cstackCOMMON 0071
start                      init         0000
start@i                    cstackCOMMON 0074
start@x                    cstackCOMMON 0070
start_initialization       cinit        0002
wtemp0                     (abs)        007E
